:100000009128A2003B200C080D0403198C2886209F
:1000100084132208800664000D280E288C0A031918
:100020008D0F0B2880068C288F002408840022095D
:100030003C2084138F0803198C28F03091000E089F
:1000400080389000F03091030319910003198F0359
:1000500003198C282B283F2003010C1822088E1F1F
:1000600022088E0803190301900F382880061F28E4
:10007000392800002228FF3A841780058C280D08B3
:100080000C0403198C0A80300C1A8D060C198D068D
:100090008C188D060D0D8C0D8D0D8C288F018E000A
:1000A000FF308E07031C8F07031C8C2803308D0044
:1000B000DF305C2050288D01E83E8C008D09FC303B
:1000C000031C65288C07031862288C0764008D0FB9
:1000D00062280C186B288C1C6F2800006F28080001
:1000E000103094008D018C01930C920C031C7E281F
:1000F0000E088C070F0803180F0F8D078D0C8C0C42
:10010000910C900C940B742810088C288C098D0984
:100110008C0A03198D0A08008313031383126400E9
:1001200008008316FF3085000C30860083121E30D5
:10013000AF000530AD000530B2000130B3006400FF
:100140000B3033020318C8280630A4001030A20078
:1001500033089200930103308E008F0170209E00BF
:1001600011089F005A309E0703189F0A1E088E0030
:100170000230142002308606831686100130831266
:10018000860683160610643083124E20B30F9F2814
:1001900064000519D4298F2129188614291C86107A
:1001A0002A1806142A1C061029089200930102300E
:1001B0008E008F0170209E0011089F002A081E07E4
:1001C000A8002808033C031CED2800308A002808FA
:1001D0008207802928295429ED280630A4001030F0
:1001E000A2005A308E000130142050308E000230B0
:1001F00014207D308E00013014205A308E000230E1
:10020000142064308E00023014200130B3006400EA
:100210000330330203181C29AA30AE007830AC003A
:100220007830B100B3216430AE00A030AC00A03013
:10023000B100B321B30F072926088C0027088D00D1
:100240003F200C08A6000D08A700640026185429BA
:100250000630A4001030A2008C308E000130142033
:1002600050308E00023014207D308E00013014207A
:100270005F308E00023014200130B3006400033080
:10028000330203185329AA30AE007830AC00A030F6
:10029000B100B3216430AE00A030AC007830B100C2
:1002A000B321B30F3E29C8280630A4001030A200A5
:1002B0008C308E000130142078308E0002301420F3
:1002C0006E308E000130142064308E000230142015
:1002D0000130B30064000330330203187F29AA30D1
:1002E000AE00A030AC007830B100B3216430AE0075
:1002F0007830AC00A030B100B321B30F6A29C82810
:10030000AA30AE00A030AC00A030B100B321643000
:10031000AE007830AC007830B100B321C828AB0112
:10032000B001A901AA010130B300640033082F0213
:10033000031CA429640006199E29AB0A64008619CF
:10034000A229B00AB30F952964002D082B02031CC3
:10035000AB290130A900640032083002031CB22925
:100360000130AA0008000130B40064000B303402F0
:100370000318D3292E088C008D01063084008030AC
:1003800001202C088C008D010630840040300120B3
:1003900031088C008D0106308400203001200D30A2
:1003A0004E20B40FB529080006108316061064000D
:1003B00083128619E0290614831606108312E42995
:1003C00006108316061083128610831686106400AA
:1003D00083120619F0298614831686108312F429D5
:0E03E0008610831686108312C8286300F52944
:02400E00F53F7C
:00000001FF
